:10000000E028083033190130A300A201360884002B
:10001000340849203408800484130005FF3E331D52
:10002000A20C3319A20D32305D20A30B0828220840
:100030000314DB28A200083033190130A300A20CFE
:1000400036088400340849203408031880043C3002
:100050005D2034088004A30B1F280314DB28B31C85
:10006000DB283528B300331CDB283608840034082D
:1000700049200130A100F4305E20340880040130B2
:10008000A100F4305E2829080319DB28D620A90333
:100090004328FF3A80054C2884178005DB28831607
:1000A0009B001C141A08DB288316F83881050F39C9
:1000B000810463000F308104DB28A101E83EA00029
:1000C000A109FC30031C6728A00703186428A007B7
:1000D0000000A10F642820186D28A01C71280000C2
:1000E00071280800013EA7000A30A200A301A42045
:1000F000A70B7728240808000310A00DA10DFF3ED0
:1001000003187C282008DB280310A10CA00CFF3E5C
:10011000031884282008DB28A20001309428A200BC
:1001200006309428A2000530A80023082102031DF0
:100130009B282208200204300318013003190230E2
:100140002805031DFF30DB28A501A4011030A600FF
:10015000210DA40DA50D2208A4022308031C230FC2
:10016000A5020318BA282208A40723080318230F9E
:10017000A5070310A00DA10DA60BA8282008DB28B9
:100180001030A800A101A001A70CA60C031CCE28CA
:100190002208A00723080318230FA107A10CA00C15
:1001A000A50CA40CA80BC4282408DB288400310863
:1001B0008A003008820083130313831200000800B2
:1001C0000730990083169F018501831285018510F0
:1001D0000130542085142130C900D324A930C9002E
:1001E000D3240630C900D3241330C900D3242030CF
:1001F000C900D3246022A9220C30C900851D022920
:100200000D30C900D3240530B6000430B4000130ED
:100210003220CC301A20BE301A202F200530B600F4
:100220000430B400003032200120BE00BF010120A4
:10023000C000C1010430A9000130B000B101432069
:100240000120C7000120C6002F2043100310BF0C5F
:10025000BE0C47081C3CC80010304802031C332960
:100260001030C80239290130BE020030031C013EA3
:10027000BF024808A600A7010A30A200A301C020BF
:10028000C8004808A000A1011030A200A301A420CA
:10029000C8004008A0004108A100A301FF3092203F
:1002A000031D622943147F30BE060030BF060130B3
:1002B0004802031C5F2948080A3CC8006229BE0A9C
:1002C0000319BF0A3E08A0003F08A100A301FF30A8
:1002D0009220031D71294314BE01BF0148080A3C46
:1002E000C8000530B6000430B40001303220CC30F4
:1002F0001A2044301A202F208C30C900D3244330D8
:10030000C900D3243E08A0003F08A100A301633028
:100310008F20031D91290730C5000130C4006722DA
:100320009A290730C5000A30C400431C99290B30B4
:10033000C40067223E08A0003F08A10001307220DF
:10034000C4000F30C50067223E08A0003F08A1008E
:1003500000307220C4001730C50067221F30C5006E
:100360000C30C40067222430C5004808A000A10159
:1003700000307220C40067222C22FF30B800FF300A
:10038000B900FF30BA00FF30BB003E08A0003F08B4
:10039000A100A30120308F20031DCF29132A3E087E
:1003A000203CBE003F08031C013E003CBF00013062
:1003B000CF004F08A000A1013F08A3003E088C20F9
:1003C000031DE6290310B80DCF0FD9290930CF003E
:1003D0004F08A000A1013F08A3003E088C20031D88
:1003E000F5290310B90DCF0FE8291130CF004F08C0
:1003F000A000A1013F08A3003E088C20031D042A91
:100400000310BA0DCF0FF7291930CF004F08A00005
:10041000A1013F08A3003E088C20031D132A0310EE
:10042000BB0DCF0F062ACF0104304F020318212A3B
:1004300024224F08383E84000008C900D424CF0F7E
:10044000142A06305420FC28CC30C900D324413073
:100450004F07C900D3240800CA01431C312A0430C5
:10046000CA00BD30C900D3244330C900D3244A0890
:10047000C900D4244A08C900D424431C412A0130AD
:10048000CA00BD30C900D3244230C900D3244A0871
:10049000C900D4244A08C900D4240130CA00431C2E
:1004A000532A4130CA00BD30C900D3244030C900AE
:1004B000D3244A08C900D4244A08C900D424080017
:1004C0008030C900D3244030C900D3240800440838
:1004D000A600A7010730A200A301C020CB00433033
:1004E000C900D32480304507C900D3240130C2009D
:1004F000083042020318832A4B084F20C900D42435
:10050000CB0AC20F782AC901D4244430C900D324AD
:1005100080304507C900D3244408A600A70107304E
:10052000A200A301C020BC002508BD005B303C0731
:10053000CB000130C200083042020318A62A4B0843
:100540004F20C900D424CB0AC20F9B2AC901D4244E
:100550000800B630CF00F5304F020318B52A4F0817
:100560004F20C900D424CF0FAB2ACF01C3304F0294
:100570000318C72B4F08C23C031CC42BC122C9005F
:0A058000C42B03308A004F08002B43
:1006000082070134A13411345134A1340134E1346E
:1006100011341134E13401348134413441344134F2
:1006200081340134013401340134FF34FF340034A7
:100630000034FF340034403458345434523451348C
:100640004034503440344F34503450344F344034BC
:100650008034FF3400340034003400340F340F345D
:100660000F34003400340034033407340F340D34B5
:100670000D340D34053400340F340F340F3400348E
:100680000F340F340F3400340F340F340F34003470
:100690003F343F343F3404340F340F3407340034D4
:1006A0000C340C34003400340034043484344534C5
:1006B000453484340434843445344534843400343B
:1006C000FF34003400340034FF3400348434043404
:1006D0000034FF34FF34003400340034E134F234A9
:1006E00012341234123412341234123412341234DA
:1006F00012341234123413341334133410341034CB
:100700000834043402340134013401340134013436
:100710000134013401340134013401340134013431
:100720000134013401340134013401340134013421
:100730008134813481340134013401340134013491
:1007400001340134013401340134FE340034003406
:100750000034103414341634153414341034133473
:100760001434143413340034FF34003400340034AF
:10077000FF340034103410340034FF34FF340034BC
:1007800000340034FF34FF34D424CF0FB62AC9011B
:100790000130CF0029304F020318D12BD424CF0FC2
:1007A000CA2BCF01CE304F020318D22C4F08CD3CBC
:1007B000031CCF2CDD23C900CF2C04308A004F0846
:0207C000002C0B
:100800008207033402340334003400343E3441346C
:10081000413441342334003400340034FF34003494
:10082000003400344034403441345F344034403488
:100830004E34513451344E340034FF3400340034DB
:100840000034FF340034423440340034FF34FF3489
:10085000003400340034FF34FF34003400340034FA
:1008600000340034003400340034003400340034E8
:1008700000340034003400340034003400340034D8
:1008800000340034003400340034003400340034C8
:1008900000340034003400340034003400340034B8
:1008A00000340034003400340034003400340034A8
:1008B0000034003400340034003400340034003498
:1008C00000340034FF340034003400340034003489
:1008D0000034003400340034383444344434383480
:1008E0000034FF34003400340034FF340034083462
:1008F00000340034FF34FF34803480348034833457
:10090000833483348334833483348334833483342F
:10091000833483348334833483348334833483341F
:10092000833483348334833483348334833483340F
:1009300083348334833483348334833483348334FF
:1009400083348334833483348334833483348334EF
:1009500083348334833483348334833483348334DF
:1009600083348334833483348334833481348034D4
:1009700080348034813481348134813481348134D1
:1009800081348134813481349E34BF34BF34BF34E8
:10099000BF34BF349E34813481348034FF34D42456
:1009A000CF0FD22B080005100130CE0009304E02C7
:1009B0000318E42CC91B0516C91F05120310C90D25
:1009C00085168512CE0FD62C051408006300E62C80
:02400E00FC3F75
:10420000FC00FE00070003000700FE00FC000000A9
:1042100000000400FF00FF00000000000C000E0082
:104220008700C300E7007E003C000C000E00070082
:104230004300E700FE00BC00C000F0003C00FF00AF
:10424000FF00000000003F003F0033003300730018
:10425000E300C300F800FC00EE006700E300C300C9
:104260008000030003008300E300FB003F000F0019
:10427000BC00FE00F7006300F700FE00BC003C003D
:104280007E00E700C300E700FE00FC000000C00065
:10429000C000F000F000C000C0000000C000C0007E
:1042A000C000C000C000C00000000000000000000E
:1042B00000000000000007000F001C0018001C0098
:1042C0000F0007000000000018001F001F0018006A
:1042D00000001E001F001B00190018001800180025
:1042E00006000E001C0018001C000F00070007004D
:1042F0000700060006001F001F00060006000E0053
:104300001C0018001C000F00070007000F001C0015
:1043100018001C000F000700000000001F001F0015
:1043200000000000000007000F001C0018001C0027
:104330000F0007000000180018001C000E00070006
:104340000300000000000000030003000000000064
:104350000000000000000000000000000000180045
:10436000180000000000000000000000FF00010035
:104370000100E1001100090089004900490089009D
:104380000900090009008900490049008900090065
:104390001100E1000100190019001900F900F900ED
:1043A000F9001900190019008100C100E100210085
:1043B000E100E100C1000100E100E100E100410095
:1043C000E100E100C1006100E100E100C100010085
:1043D000E100E100E1004100E100E100C100010075
:0A43E00001000100010001000100CE
:00000001FF
